:1000000002C10000ABC600007EC6000051C6000061
:1000100024C60000F7C50000CAC5000024C10000C6
:1000200022C1000020C100001EC100001CC1000050
:100030001AC1000018C1000016C1000014C1000060
:1000400012C1000010C100000EC100000CC1000070
:100050000AC1000008C1000006C100005EC5000022
:1000600002C1000024C50000F9C40000FCC000006B
:10007000FAC00000F8C00000F6C00000F4C00000A4
:10008000F2C00000F0C00000EEC00000ECC00000B4
:10009000EAC00000E8C00000E6C00000E4C00000C4
:1000A000E2C00000E0C00000DEC00000DCC00000D4
:1000B000DAC00000D8C00000D6C00000D4C00000E4
:1000C000D2C00000D0C00000CEC00000CCC00000F4
:1000D000CAC00000C8C00000C6C00000C4C0000004
:1000E000C2C00000000020002300260029002C00D0
:1000F0002F00320000010000030106010901000089
:100100002100240027002A002D00300033000101C7
:100110000000040107010A01000022002500280058
:100120002B002E00310034000201000005010801FF
:100130000B0105050505070508080808020202026B
:100140000A0A080804040404010101010101010173
:100150000303030303030303040707070C0C0C0C3E
:100160000C0C0C0C02020202060606060606060627
:100170000B0B0B0B0B0B0B0B0102102020080810B4
:100180002040102040800201020108040201010207
:1001900004081020408080402010080402018004E0
:1001A000020180402010080402010804020101023B
:1001B0000408102040800102040810204080000044
:1001C0000A0B02090C0D0E080703040100000000D1
:1001D000000000000000000000000000000000001F
:1001E00000000000000000000000121110000000DC
:1001F00000000000000000000000000000000000FF
:1002000000000000A80711241FBECFEFD1E2DEBF1F
:10021000CDBF00E00CBF27E0A8E5B4E001C01D920F
:10022000A430B207E1F714E0A0E0B2E0EEE4FBE1B5
:1002300000E00BBF02C007900D92A835B107D9F7B7
:1002400011E0C3E0D1E000E006C021970109802F52
:10025000FE010E94740CC230D10780E00807A9F7A4
:100260000AD70C94A50DCCCEAF92BF92CF92DF925D
:10027000EF92FF920F931F93CF93DF936C017B015B
:100280008B01040F151FEB015E01AE18BF08C017EC
:10029000D10759F06991D601ED91FC910190F0815F
:1002A000E02DC6011995892B79F7C501DF91CF9112
:1002B0001F910F91FF90EF90DF90CF90BF90AF9084
:1002C0000895FC01538D448D252F30E0842F90E05C
:1002D000821B930B541710F0CF9608950197089541
:1002E000FC01918D828D981761F0A28DAE0FBF2F0A
:1002F000B11D5D968C91928D9F5F9F73928F90E060
:1003000008958FEF9FEF0895FC01918D828D9817CE
:1003100031F0828DE80FF11D858D90E008958FEF0B
:100320009FEF0895FC01918D228D892F90E0805CD4
:100330009F4F821B91098F739927089585EE94E052
:10034000F1DF21E0892B09F420E0822F0895FC01E0
:10035000A48DA80FB92FB11DA35ABF4F2C91848D26
:1003600090E001968F739927848FA689B7892C9383
:10037000A089B1898C91837080648C93938D848DD6
:10038000981306C00288F389E02D80818F7D8083D9
:100390000895EF92FF920F931F93CF93DF93EC0199
:1003A00081E0888F9B8D8C8D98131AC0E889F9891C
:1003B000808185FF15C09FB7F894EE89FF8960831F
:1003C000E889F98980818370806480839FBF81E0A0
:1003D00090E0DF91CF911F910F91FF90EF900895E2
:1003E000F62E0B8D10E00F5F1F4F0F731127E02EBD
:1003F0008C8D8E110BC00FB607FCFACFE889F989F6
:10040000808185FFF5CFCE01A2DFF2CFEB8DEC0F1F
:10041000FD2FF11DE35AFF4FF0829FB7F8940B8F29
:10042000EA89FB8980818062D0CFCF93DF93EC0192
:10043000888D8823B1F0AA89BB89E889F9898C91D4
:1004400085FD03C0808186FD0CC00FB607FCF7CF89
:100450008C9185FFF2CF808185FFEDCFCE0177DFD4
:10046000EACFDF91CF9108958150823108F05AC0D0
:10047000E82FF0E08827E05CFD4F8F4F0C94740C60
:1004800060026402520258025C02920267026D022C
:10049000710277027B027F028502890292028D023D
:1004A00093029702809180008F7780938000089557
:1004B000809180008F7DF9CF80918000877FF5CF7C
:1004C00084B58F7784BD089584B58F7DFBCF8091EF
:1004D000B0008F778093B00008958091B0008F7D39
:1004E000F9CF809190008F7780939000089580914C
:1004F00090008F7DF9CF80919000877FF5CF80911C
:10050000A0008F778093A00008958091A0008F7D38
:10051000F9CF8091A000877FF5CF809120018F7760
:10052000809320010895809120018F7DF9CF8091E3
:100530002001877FF5CF1F93CF93DF93282F30E0E3
:10054000F901E254FE4F8491F901E858FE4FD4912D
:10055000F901EE5CFE4FC491CC23A1F0162F81115E
:1005600083DFEC2FF0E0EE0FFF1FE85EFE4FA5915A
:10057000B4918FB7F894EC91111108C0D095DE2397
:10058000DC938FBFDF91CF911F910895DE2BF8CFC1
:10059000CF93DF9390E0FC01E858FE4F24918E5CEE
:1005A0009E4FFC0184918823C9F090E0880F991F29
:1005B000FC01E250FF4FA591B491FC01E85EFE4FB3
:1005C000C591D49161110DC09FB7F8948C9120957D
:1005D00082238C938881282328839FBFDF91CF912A
:1005E0000895623051F49FB7F8943C91822F809522
:1005F00083238C93E8812E2BEFCF8FB7F894EC9167
:100600002E2B2C938FBFEACF3FB7F8948091CF0465
:100610009091D004A091D104B091D20426B5A89BAA
:1006200005C02F3F19F00196A11DB11D3FBFBA2F84
:10063000A92F982F8827BC01CD01620F711D811D44
:10064000911D42E0660F771F881F991F4A95D1F7C9
:1006500008958F929F92AF92BF92CF92DF92EF92C6
:10066000FF924B015C01D0DF6B017C01CDDF6C1987
:100670007D098E099F09683E734081059105B0F39D
:1006800021E0821A9108A108B10888EEC80E83E023
:10069000D81EE11CF11C81149104A104B10431F7AE
:1006A000FF90EF90DF90CF90BF90AF909F908F9092
:1006B00008952FB7F8946091CB047091CC04809189
:1006C000CD049091CE042FBF0895FC01848187FD55
:1006D00004C091E0692763832EDF80E00895FC0168
:1006E000808580FD04C082FB882780F9089580E022
:1006F0000895FC019085957081E0953009F080E0C7
:100700000895862F642F44CFCF93DF93FC0121857A
:1007100030E0F901E254FE4F8491F901E858FE4FB0
:10072000D491F901EE5CFE4FC491CC2371F081119C
:100730009BDEEC2FF0E0EE0FFF1FEC51FF4FA59179
:10074000B491EC91ED2381E009F480E08170DF91B8
:10075000CF9108950F931F93CF93DF9385EE94E08D
:10076000E1DD892BA1F185EE94E0BADD8C3329F42B
:100770001092C9041092C804F1CF8A30B1F4C0E2DB
:10078000D2E004E614E089919991009739F0F801DC
:10079000208161E0213309F060E0CDDE0F5F1F4F63
:1007A000F2E0C433DF0779F7E3CF2091C80430913A
:1007B000C90424363105E4F6F901EC59FB4F808376
:1007C0002F5F3F4F3093C9042093C804C7CFDF91F8
:1007D000CF911F910F910895B1DD8111BBDF80E0B2
:1007E00090E0892B49F080E090E0892B29F00E946D
:1007F000000081110E94000080E090E0892B49F008
:1008000080E090E0892B29F00E94000081110E9475
:10081000000080E090E0892B49F080E090E0892B97
:1008200029F00E94000081110C9400000895DC0161
:10083000ED91FD918081ED91FD919081ED91FD9182
:100840006C9163708E2309F064609F2309F06860E7
:10085000E4E3F4E0E60FF11D659565956D936D9108
:100860007D918D919D91099423C01AC012C016C02C
:1008700010C01EC009C014C013C006C019C009C0F2
:100880000DC007C00DC014C0625070408040904041
:100890000BC0615070408040904006C06E5F01C048
:1008A0006F5F7F4F8F4F9F4F9E938E937E936E937C
:1008B0000895CF93DF93EC018B85823058F4F89440
:1008C000CE01B5DF6F81788589859A857894DF912F
:1008D000CF910895F894F6CFCF92DF92EF92FF92E6
:1008E0000F931F93CF93DF93EC01E62E84E090E00B
:1008F0000E947C0CFC0184E6808385E6818386E689
:10090000828387E6838380E992E0998388838FEFEF
:100910008A838B838C838A878B878C8784E0898703
:100920008F016E0185E0C80ED11CF12CF801819178
:100930008F0187FD32C0F60181936F0161E028DEEF
:10094000F394F4E0FF12F2CF8FEF8C8386E992E00C
:10095000998388838B8587FD0FC0282F082E000C74
:10096000330BE216130641F09A85913011F460E0E2
:10097000E2DD60E08B850CDE82E08A87EB8662E058
:100980008E2D06DE81E08C87DF91CF911F910F9134
:10099000FF90EF90DF90CF900895F986D5CF8F929A
:1009A0009F92AF92BF920F931F93CF93DF93CDB7D8
:1009B000DEB7A1970FB6F894DEBF0FBECDBF19A268
:1009C000423008F44AE08E010F5D1F4F842E912CB7
:1009D000B12CA12CA501940149D7E62FB901CA0178
:1009E000EA303CF5E05DD801EE938D01232B242BFA
:1009F000252B81F790E080E0109761F0FD010190D8
:100A00000020E9F73197AF014A1B5B0BBD0185EE72
:100A100094E02ADCA1960FB6F894DEBF0FBECDBFDE
:100A2000DF91CF911F910F91BF90AF909F908F90CA
:100A30000895E95CD8CF009761F0FC010190002097
:100A4000E9F73197AF01481B590BBC0185EE94E0E3
:100A50000BCC90E080E008950E94A10D1F920F92B0
:100A60000FB60F9211240BB60F922F933F934F9313
:100A70005F936F937F938F939F93AF93BF93EF9306
:100A8000FF9385EE94E063DCFF91EF91BF91AF910E
:100A90009F918F917F916F915F914F913F912F9196
:100AA0000F900BBE0F900FBE0F901F9018951F92C6
:100AB0000F920FB60F9211240BB60F922F938F93B4
:100AC0009F93EF93FF93E091F504F091F6048081FA
:100AD000E091FB04F091FC0482FD1DC090818091A7
:100AE000FE048F5F8F732091FF04821741F0E09125
:100AF000FE04F0E0EB51FB4F958F8093FE04FF91D5
:100B0000EF919F918F912F910F900BBE0F900FBE81
:100B10000F901F9018958081F2CF1F920F920FB601
:100B20000F9211242F933F938F939F93AF93BF9373
:100B30008091CB049091CC04A091CD04B091CE04CF
:100B40003091CA0423E0230F2D3758F50196A11DDB
:100B5000B11D2093CA048093CB049093CC04A0933E
:100B6000CD04B093CE048091CF049091D004A09195
:100B7000D104B091D2040196A11DB11D8093CF0480
:100B80009093D004A093D104B093D204BF91AF91BD
:100B90009F918F913F912F910F900FBE0F901F90BB
:100BA000189526E8230F0296A11DB11DD2CF1F92E2
:100BB0000F920FB60F9211240BB60F922F933F9303
:100BC0004F935F936F937F938F939F93AF93BF9355
:100BD000EF93FF9380915A0490915B0428DEFF917C
:100BE000EF91BF91AF919F918F917F916F915F91A5
:100BF0004F913F912F910F900BBE0F900FBE0F9012
:100C00001F9018951F920F920FB60F9211240BB6DA
:100C10000F922F933F934F935F936F937F938F9395
:100C20009F93AF93BF93EF93FF938091580490915C
:100C30005904FDDDFF91EF91BF91AF919F918F918D
:100C40007F916F915F914F913F912F910F900BBECC
:100C50000F900FBE0F901F9018951F920F920FB616
:100C60000F9211240BB60F922F933F934F935F93E4
:100C70006F937F938F939F93AF93BF93EF93FF9364
:100C80008091620490916304D2DDFF91EF91BF9156
:100C9000AF919F918F917F916F915F914F913F9114
:100CA0002F910F900BBE0F900FBE0F901F901895B5
:100CB0001F920F920FB60F9211240BB60F922F9323
:100CC0003F934F935F936F937F938F939F93AF93D4
:100CD000BF93EF93FF938091600490916104A7DD2F
:100CE000FF91EF91BF91AF919F918F917F916F9104
:100CF0005F914F913F912F910F900BBE0F900FBEC0
:100D00000F901F9018951F920F920FB60F921124FB
:100D10000BB60F922F933F934F935F936F937F93F5
:100D20008F939F93AF93BF93EF93FF9380915E0454
:100D300090915F047CDDFF91EF91BF91AF919F9106
:100D40008F917F916F915F914F913F912F910F9074
:100D50000BBE0F900FBE0F901F9018951F920F9211
:100D60000FB60F9211240BB60F922F933F934F9310
:100D70005F936F937F938F939F93AF93BF93EF9303
:100D8000FF9380915C0490915D0451DDFF91EF91A0
:100D9000BF91AF919F918F917F916F915F914F9193
:100DA0003F912F910F900BBE0F900FBE0F901F9091
:100DB000189590E0823090F404968330910569F1A3
:100DC0007CF481309105C9F00297F9F080916900B7
:100DD0008C7F816080936900E89A08950297EDCF37
:100DE0008430910511F1059789F780916A00837F1E
:100DF000846080936A00ED9A089580916900837FF2
:100E0000846080936900E99A0895809169008F7CDD
:100E1000806180936900EA9A0895809169008F73D8
:100E2000806480936900EB9A089580916A008C7FBA
:100E3000816080936A00EC9A0895823161F130F408
:100E4000823079F08330A9F080E008958431B9F0E0
:100E5000E0F08531C9F770935D0460935C0482E033
:100E600005C0709359046093580480E0A2DF81E0CC
:100E7000089570935B0460935A0481E0F7CF7093F8
:100E80005F0460935E0483E0F1CF7093610460932C
:100E9000600484E0EBCF709363046093620485E0A8
:100EA000E5CF0F931F93CF93DF93EC01062F142F01
:100EB00062E0802F6DDB62E0812F6ADB802F90E0A3
:100EC000FC01EE5CFE4FE491F0E0EE0FFF1FEC51F1
:100ED000FF4FA591B491B983A883FC01E858FE4F58
:100EE00024912C83812F90E0FC01EE5CFE4FE49175
:100EF000F0E0EE0FFF1FEC51FF4F459154915B83E3
:100F00004A83FC01E858FE4FE491ED831F82188666
:100F100019861A868BE39FE10197F1F78C912823BC
:100F200091E009F490E0DA018C91E82309F09260F5
:100F30009E83BE01802F81DF8B87BE01812F7DDFE5
:100F40009B85890F8B87DF91CF911F910F9108951A
:100F50001092E8041092E70488EE93E0A0E0B0E07D
:100F60008093E9049093EA04A093EB04B093EC041B
:100F70008CE992E09093E6048093E50485EC90E0A0
:100F80009093F2048093F10484EC90E09093F40445
:100F90008093F30480EC90E09093F6048093F50442
:100FA00081EC90E09093F8048093F70482EC90E059
:100FB0009093FA048093F90486EC90E09093FC04FB
:100FC0008093FB041092FE041092FF04109200051F
:100FD0001092010562E683EF96E07EDC63E686EE22
:100FE00096E07ADC42E063E186EB96E05ADF82EB42
:100FF00092E09093C3068093C2068FEB92E09093A9
:10100000C5068093C40643E269E286EC96E049DFB8
:101010008CEC92E09093D3068093D20683ED92E01D
:101020009093D5068093D40647E265E286ED96E07C
:1010300038DF8AED92E09093E3068093E20682EE39
:1010400092E09093E5068093E406E2E8F5E02EEA6C
:1010500032E08AE090E0318320831282138214828E
:10106000158297838683108611863E9646E0E63B7E
:10107000F40789F70895CF93DF9300D01F92CDB77F
:10108000DEB7789484B5826084BD84B5816084BD08
:1010900085B5826085BD85B5816085BD80916E0016
:1010A000816080936E001092810080918100826047
:1010B0008093810080918100816080938100809184
:1010C00080008160809380008091B1008460809373
:1010D000B1008091B00081608093B0008091910058
:1010E0008260809391008091910081608093910053
:1010F000809190008160809390008091A100826037
:101100008093A1008091A10081608093A1008091D3
:10111000A00081608093A000809121018260809373
:101120002101809121018160809321018091200122
:1011300081608093200180917A00846080937A009E
:1011400080917A00826080937A0080917A00816039
:1011500080937A0080917A00806880937A00109260
:10116000C10022E835E03A83298304E312E04AE033
:10117000C42ED12CD801FC9011967C91A981BA8102
:10118000ED91FC9111970280F381E02D42E050E057
:101190006F2DCD011995E981FA81F1861086DF0165
:1011A0000190F081E02D0190F081E02DCD011995A5
:1011B000882329F0E981FA8180858360808779DA44
:1011C000A981BA8112966D937D938D939C93159707
:1011D0001796DC92CE9216970C5F1F4F1E96BA831D
:1011E000A983A65BB64031F686EB96E062DB60939E
:1011F000D9047093DA048093DB049093DC0486ECCA
:1012000096E057DB6093DD047093DE048093DF0487
:101210009093E00486ED96E04CDB6093E1047093DC
:10122000E2048093E3049093E40400E212E01A8362
:101230000983A981BA81ED90FD90BA83A983E11455
:10124000F10431F061E08E2DA3D961E08E2D73D9C8
:10125000E981FA81E453F24061F768E873E180E0E4
:1012600090E0F7D9D8018D919D918D01009711F0F3
:1012700060E061D929803A802016310699F7E09123
:10128000F504F091F60482E08083E091F104F0919E
:10129000F2041082E091F304F091F40480E1808381
:1012A0001092FD04E091F904F091FA0486E0808345
:1012B000E091F704F091F804808180618083E091EF
:1012C000F704F091F804808188608083E091F7044E
:1012D000F091F804808180688083E091F704F091B8
:1012E000F80480818F7D808382E390E0A0E0B0E00D
:1012F0008093E9049093EA04A093EB04B093EC0488
:101300008AEE92E06624639422E08D3F920721F0FA
:101310008351934009F0612CCCD94B015C01809141
:10132000160290911702A0911802B0911902AC0117
:10133000BD014854544F6F4F7F4F84169506A60643
:10134000B70628F488169906AA06BB0640F589E276
:1013500093E071DB8AEE92E06EDB88E393E06BDB77
:101360004AE065E070E080E090E019DB88E393E01C
:1013700062DB80E192E05FDB8FE793E05CDB8092F1
:10138000160290921702A0921802B092190280924F
:101390000C0290920D02A0920E02B0920F0226EB68
:1013A000222E26E0322E39ED432E34E0532E10E06B
:1013B00000E0772473948AEE92E08A53934009F018
:1013C000712CF10184859585F3E08D349F0709F434
:1013D00009C18855934009F405C1D1011E968D912C
:1013E0009C9121E0B3E083369B0721F08E56934019
:1013F00009F020E0C101772009F4F6C0222309F4A6
:10140000F3C057DA24E030E040E050E051D2690107
:101410007A01F20180819181A281B3818C159D05B1
:10142000AE05BF050CF0EBC021E08091D704909190
:10143000D804019709F020E0272109F4DBC001302E
:10144000110509F0D7C08091F4069091F506F3DA02
:101450008FE793E0F0DA80920C0290920D02A09256
:101460000E02B0920F02D201CD92DD92ED92FD926A
:101470002D010F5F1F4FB0E12B0E311C0330110502
:1014800009F097CF94E3C92E92E0D92EE2E8F5E077
:10149000FA83E983F12CE12CA981BA8118968C9109
:1014A00018978B7F18968C931897ED91FC91119754
:1014B0000190F081E02DCD011995182FE981FA8175
:1014C000808586958170181709F4B5C0F2D8A98176
:1014D000BA8112966D937D938D939C931597189670
:1014E0008C91B2E08B27E981FA81808789819A818A
:1014F000F6D8811106C089819A81FBD8882309F426
:101500005FC0D6010D911C91C801039783309105EE
:1015100090F00431110579F04097039708F4C6C0A4
:1015200081E00C31110509F080E0662009F4C0C0AB
:10153000882309F4BDC08092080290920902A0920B
:101540000A02B0920B021092D6041092D504D60172
:1015500012968D919C916FDA89819A81C0D88823E7
:1015600009F471C189E793E066DA0B321105D9F409
:101570007720C9F08091D7049091D804009709F0A2
:1015800059C1E1E0F0E0F093D804E093D7048092F1
:10159000000290920102A0920202B092030261E066
:1015A00080E00E949B0264E670E080E090E051D809
:1015B00080920C0290920D02A0920E02B0920F0245
:1015C000FFEFEF1AFF0A29813A81225F3F4F3A83EA
:1015D000298334E0C30ED11C46E1E416F10409F07E
:1015E0005BCF93C021E006CF64D922E030E040E039
:1015F00050E00CCFD1011E968D919C9128CFC8163A
:10160000D906EA06FB060CF02ECF21E08091D70424
:101610009091D804019709F020E0272141F0013092
:10162000110529F48091F2069091F30610CFF10193
:10163000848595850CCF3DD8A981BA8112962D91CC
:101640003D914D915C9115971B012C01221A330A93
:10165000440A550AB201A10116968D919C91B0E001
:10166000A0E0481759076A077B0708F43FCFA98114
:10167000BA8118968C918170181709F437CF19D850
:10168000E981FA8162837383848395838085F1E0A5
:101690008F278460A981BA8118968C930AD8E98132
:1016A000FA81628773878487958720CF81E03DCF59
:1016B0000231110539F00A31110509F048CF6620D1
:1016C00009F445CF8091080290910902A0910A0285
:1016D000B0910B0286509F4FAF4FBF4F88169906AF
:1016E000AA06BB0690F0E1E0F0E0F093D604E093A8
:1016F000D504F092D404E092D30480920402909234
:101700000502A0920602B09207028AEE92E08A5386
:10171000934001F58091000290910102A091020294
:10172000B091030288539D4CAF4FBF4F8815990568
:10173000AA05BB0520F41092D8041092D70480911A
:10174000D7049091D80460E0892B09F061E080E033
:101750000E949B0280910C0290910D02A0910E02BA
:10176000B0910F02AC01BD014C595F4F6F4F7F4FDD
:1017700084169506A606B70628F488169906AA06C2
:10178000BB0658F48FE793E056D980920C029092F2
:101790000D02A0920E02B0920F028091040290916D
:1017A0000502A0910602B091070286509F4FAF4FED
:1017B000BF4F88159905AA05BB05C8F58091D504CA
:1017C0009091D604019799F5E091D304F091D40457
:1017D000EE0FFF1FEE0FFF1FEC5CFD4F8281938128
:1017E0002AD98091D3049091D404BEE0B89F80019F
:1017F000B99F100D11240E571A4FC8010E946F0394
:10180000882361F189E793E016D964E670E080E00F
:1018100090E00E94290380920C0290920D02A09207
:101820000E02B0920F021092D6041092D5040E94BC
:10183000EC0372CD019709F0B6CE1092D804109245
:10184000D70460E0ADCE89819A810E947903882314
:1018500009F4A9CE8DE793E0EED8A5CEC8010E9489
:101860007903882391F28DE793E0CECFA1E21A2E7F
:10187000AA1BBB1BFD010DC0AA1FBB1FEE1FFF1F34
:10188000A217B307E407F50720F0A21BB30BE40B84
:10189000F50B661F771F881F991F1A9469F76095CB
:1018A0007095809590959B01AC01BD01CF01089585
:1018B000052E97FB16F400940FD057FD05D0D6DF08
:1018C00007FC02D046F408C050954095309521950C
:1018D0003F4F4F4F5F4F089590958095709561955C
:1018E0007F4F8F4F9F4F0895EE0FFF1F881F8BBFB5
:1018F0000790F691E02D19940F931F93CF93DF93E8
:101900008230910510F482E090E0E0910207F091BE
:10191000030730E020E0B0E0A0E0309799F4211513
:10192000310509F44AC0281B390B24303105D8F59C
:101930008A819B816115710589F1FB019383828303
:10194000FE0111C04081518102811381481759075E
:10195000E0F04817590799F4109761F012960C932C
:10196000129713961C933296CF01DF91CF911F915E
:101970000F9108950093020710930307F4CF2115E8
:10198000310551F04217530738F0A901DB019A01E4
:10199000BD01DF01F801C1CFEF01F9CF909303073B
:1019A00080930207CDCFFE01E20FF31F8193919345
:1019B0002250310939832883D7CF209100073091F5
:1019C0000107232B41F420911C0230911D0230931A
:1019D00001072093000720911A0230911B02211564
:1019E000310541F42DB73EB740911E0250911F02C0
:1019F000241B350BE0910007F0910107E217F30774
:101A0000A0F42E1B3F0B2817390778F0AC014E5F6E
:101A10005F4F2417350748F04E0F5F1F50930107A3
:101A200040930007819391939FCFF0E0E0E09CCF3B
:101A3000CF93DF930097E9F0FC0132971382128273
:101A4000A0910207B0910307ED0130E020E010976C
:101A5000A1F420813181820F931F209100073091E2
:101A600001072817390709F061C0F0930107E093D7
:101A70000007DF91CF910895EA01CE17DF07E8F55F
:101A80004A815B819E0141155105B1F7E901FB8354
:101A9000EA8349915991C40FD51FEC17FD0761F4F2
:101AA000808191810296840F951FE9019983888333
:101AB000828193819B838A83F0E0E0E012968D918E
:101AC0009C9113970097B9F52D913C911197CD01F9
:101AD0000296820F931F209100073091010728176B
:101AE000390739F6309751F5109203071092020723
:101AF000B0930107A0930007BCCFD383C28340817A
:101B00005181840F951FC817D90761F44E5F5F4F4D
:101B100088819981480F591F518340838A819B8115
:101B2000938382832115310509F0B0CFF093030729
:101B3000E09302079ECFFD01DC01C0CF1382128229
:0E1B4000D7CF81E090E0F89400C0F894FFCF7A
:101B4E00FFFFFFFFFFFFFFFFFFFFFFFFFFFFFFFF97
:101B5E00322E362E3200FFFFFFFF000004078000FA
:101B6E002E0010001600190017002D001B001D007E
:101B7E0018000F003500810334008A031F00930301
:101B8E002A009C033300A5033200AE030E00B703F8
:101B9E002000BF031C00C9031E00D2031A00DB0382
:101BAE002400E4032200ED032600F7032800FF03C0
:101BBE002C0009043000110403001A04140025043B
:101BCE000500330404003E0412004B040000000024
:101BDE002C0500000000650300000000C90134015F
:101BEE00610115029201700184010000000084035E
:101BFE008103454E435F52414E47455F444E00457B
:101C0E004E435F52414E47455F555000564F4C5F15
:101C1E00444E00564F4C5F555000435253525F4452
:101C2E004E00435253525F5550005265616C5369DA
:101C3E006D476561722D474D4133353000526561F8
:101C4E006C53696D476561722D47313030305046A7
:101C5E004431005265616C53696D476561722D4761
:101C6E00313030304D4644310023232323526561F9
:101C7E006C53696D4765617223005265616C5369DF
:101C8E006D476561722D47464335303000454E43F2
:101C9E005F4844475F555000454E435F414C545F8B
:101CAE00555000454E435F4844475F444E00454EF5
:101CBE00435F414C545F444E003D310A003D300AB3
:101CCE000042544E5F4D4943310042544E5F4D49E0
:101CDE0043320042544E5F4E4156310042544E5FE5
:101CEE004E4156320042544E5F434F4D31004254E6
:101CFE004E5F434F4D320042544E5F4D4B520042A9
:101D0E00544E5F4D414E53510042544E5F53504B13
:101D1E00520042544E5F4D5553320042544E5F5066
:101D2E004153530042544E5F4D5553310042544E71
:101D3E005F434F504C540042544E5F54454C00424A
:101D4E00544E5F50494C4F540042544E5F415558CB
:101D5E000042544E5F504C41590042544E5F504128
:101D6E004E5F444E0042544E5F50414E5F524947C3
:101D7E0048540042544E5F50414E5F5550004254FD
:101D8E004E5F50414E5F4C4546540042544E5F509C
:081D9E00414E5F53594E430012
:00000001FF
